:03000000021CE8F7
:0C1CE80078FFE4F6D8FD7581DF020036BD
:0100190022C4
:061A02008B2C8A2D892EB9
:101A08007571027F48121B75121D2DEF20E0F9AB8E
:101A18002CAA2DA92E120A74787AE6FE08E6FDEDA6
:011A2800FFBE
:011A2900229A
:1010470043525354005341564500434647002D3EF3
:1010570053320052415445434C5220554E49544255
:101067004C4E4B545249475452455653545254537D
:10107700544F505A45524F4241554444464C54539D
:1010870041564552535420535720202E3173202E5A
:101097003273202E35732031732020327320203590
:1010A7007320203130732033307320316D2020328C
:1010B7006D2020356D202031306D2033306D20318B
:1010C7006820200000000100020005000A0014004B
:1010D700320064012C025804B00BB8177046508CCC
:1010E700A001020408103046656574596172644DA9
:1010F7006574724F6666204F6E20204E6F20205910
:101107006573204F66662054696D65416C74205481
:101117007269674F6666205472696750777220520A
:03112700656320DD
:101A750025E024CAF582E43410F58322052EE52EEF
:101A8500C3940222A62EE52E75F004A42208F608BA
:041A9500F608F62237
:10156100789A76AB0876CD08760008760AE408F614
:1015710008760108F6087664087640121A9208F691
:1015810078A8F608760A08F608763C08F608761474
:1015910008F608760F121A9278B576057BFF7A1055
:0D15A100794712191C7F0512187E0219AC43
:10194E0075751D7576C0121685789BE664CD70048C
:10195E0018E664AB600312156178B4E6FFF4600319
:0F196E00EF700478B4760178B5E6B4FF02760521
:01197D002247
:0D1CA200C2AF7DC07C1DE4FF121C00D2AF5C
:011CAF002212
:101685007539FF85753A85763B753C00753D007566
:101695003E9AE4FFAB39AA3AA93B8F8275830012C3
:1016A5000A47AB3CAA3DA93E8F82758300120A8684
:1016B5000FBF1CE078B3E6FFF46003EF700478B366
:0216C5007601AC
:0116C7002200
:1019AC007D01E4FF121B1D7BFF7A10794C12191C70
:1019BC00121CA2C2AF7F9A7B1C7DC07C1D121C0A1C
:0D19CC00D2AF7F0212187EE4FDFF021B1D4A
:10058300E4F52C7BFF7A10795112191C7F051218A0
:100593007EA297829650FAA296921AA297921BE590
:1005A3002C75F004A4245AF9741035F0FA7BFF1269
:1005B300191C7F0512187E852C2DE4F52E7BFF7AFE
:1005C30010795512191CE52CB40A00400302065198
:1005D3009005DAF82828730205F802065102061975
:1005E30002062102062502062D02063502063902FD
:1005F30006410206497F01EF121A75789CE6FC0852
:10060300E6FD7401936D7003E4936C70028F2E0FFB
:10061300BF0FE40206D7789EE6F52E0206FA789F0E
:10062300800278A7E6F52E02071478A6E6F52E02D7
:10063300074278B0800278B1E6F52E02075F78B200
:10064300E6F52E02079478B5E6F52E0207BAE52CF7
:10065300652D60030205A2A21A309601B35013A2BE
:1006630096921A30960C052CE52CC3940D4003E4A6
:10067300F52CA21B309701B350D4A297921B30974D
:10068300CDE52CB40D0050C6900692F828287302CD
:1006930006B90206E20206E802070602072002077D
:1006A3003402074D02076A0207820207A80207CB3A
:1006B3000207D10207D7052EE52EC3940F40037519
:1006C3002E01E52E121A75E493FF740193789CCFE3
:1006D300F608EFF6121A8B248EF9741002079D1296
:1006E30014B7020651052EE52EC394034003E4F527
:1006F3002E789EA62EE52E75F004A424EEF9741030
:1007030002079D121A814003E4F52E789FA62EE579
:100713002E75F004A424FAF9741002079D121A81AD
:100723004003E4F52E78A7121A8924FAF97410808D
:1007330069121A814003E4F52E78A6A62EE52E75DC
:10074300F004A42402F974118050052EE52EC394FD
:10075300044003E4F52E78B0A62EE52E75F004A42C
:10076300240AF974118033052EE52EC39403400344
:10077300E4F52E78B1121A89240AF97411801B0545
:100783002EE52EC394044003E4F52E78B2A62EE59D
:100793002E75F004A4241AF9741135F0FA7BFF12B4
:1007A300191C020651052EE52EC394064003E4F5F9
:1007B3002E78B5A62EE52E9010E89375F018A4FFB9
:1007C300AEF012127C020651121561020651121983
:0A07D300AC02065143A208020651D1
:0A1D00004552415300444F4E450088
:101C6300789CE6F54F08E6F55022E566AE65780602
:011C7300224E
:1011F000C218C21978B4E6FFE4FCFDFEFB7A20F9C0
:10120000F8120AA88F6C8E6B8D6A8C69E47B40FAA9
:10121000F9F8120B338E638F64E4F52DF52EC3E5D8
:101220002E9564E52D9563501CE52C64816016AF06
:101230002EAE2D12197E121BEC8F2C052EE52E7072
:10124000DD052D80D9E52CB48108E52E152E700220
:10125000152DE52E65647004E52D6563700CD218BC
:10126000121CCCE4F565F5668007852D65852E6634
:0B127000E4F567F568754E80121C6302
:01127B002250
:10197E00C3EF9564EE95635024EF7806C333CE33F0
:10198E00CED8F9FD757102EE787AF6CFEDCFEF086D
:0D199E00F67F50121BAA121D2DEF20E0F95C
:0119AB002219
:031B9000CDEFCDC9
:101B9300757102EE787AF6ED08F67F50121BAA12E1
:061BA3001D2DEF20E0F90A
:011BA9002219
:101BEC007571017F50121B75121D2DEF20E0F978D5
:031BFC007AE6FF87
:011BFF0022C3
:101BD700121B90E4FFFE0FBF00010EBE0FF8BFA05F
:041BE700F5121BECEC
:011BEB0022D7
:0618B400CBEFCBCAEECA27
:1018BA00301803301927757103EA787AF6EB08F6BF
:1018CA0008EDF67F50121BAA121D2DEF20E0F9E455
:0D18DA00FFFE0FBF00010EBE0FF8BFA0F50E
:0118E70022DE
:10170B00752F0075300075314EE4F52E121C6DC32C
:10171B0033CE33CED8F97C00252EFFEC3EFEAB2F1B
:10172B00AA30A931852E82758300120A47FD121843
:10173B00B4052EE52EC3940640D275670075680676
:01174B00227B
:101382008E2C8F2D121C6DC333CE33CED8F9256827
:10139200FFE5673EFEEEC0E0EFC0E0E52CFDD0E0E9
:1013A200FFD0E0FE1218B40568E568700205671206
:1013B2001C6DC333CE33CED8F92568FFE5673EFEF8
:1013C200AD2D1218B40568E568700205670552E58F
:1013D2005270020551C3E5689440E56794004017D6
:1013E200E4F567F5680566E566700205659564E5EE
:0813F2006595634002D2182248
:1014B700E4F567F5687BFF7A1D790012191CD219CC
:1014C700E4F539F53AC3E53A9564E5399563502172
:1014D700E53AAE397806C333CE33CED8F9F5688E00
:1014E700677D81FF1218B4053AE53A70D80539804F
:1014F700D4C2197BFF7A1D790512191CE4F565F52D
:0715070066F567F568C218E4
:01150E0022BA
:10145E00E4F539F53AF53BF53CC3E53C9564E53BDF
:10146E0095635044E53A6481603EAF3CAE3B121941
:10147E007E121BEC8F3AE53A64807022AF39053943
:10148E00FCFDFEFBFAF9120E1E7F2C120016AE3B6F
:10149E00AF3CE4FCFDFBFAF9120E1E121D1D053CBD
:0814AE00E53C70B5053B80B17F
:0114B6002213
:0215FA008F3927
:1015FC00E4F53AF53BF53CF53DC3E53D9564E53C3A
:10160C0095635030E53B6481602AAF3DAE3C1219C6
:10161C007E121BEC8F3BE53BB4800FE53A653970CD
:10162C0007AF3DAE3C02197E053A053DE53D70C95C
:04163C00053C80C524
:011640002287
:10174C00121C6378A7E6F553E4F551F55212170B0A
:10175C0085656D85666E7F011213FA30021A78AAC0
:10176C00E6FE08E6FFE4FCFD7B64FAF9F8120AA831
:10177C008F608E5F8D5E8C5D300505C205121BC1BE
:01178C00223A
:1018440085652C85662DE56845676008052DE52DC1
:101854007002052C856D65856E6612170B852C65E7
:10186400852D66C3E52D9564E52C95634007E4F565
:0A18740065F566D2187F020213FA30
:101C0000740478FF769612FF0322740078FF7696AC
:041C100012FF03229A
:0300330002112A8D
:0D112A00C0E0C0F0C083C082C0D075D00806
:10113700E5D954F8FF120C4C1164081164101173AF
:1011470018118E20117528118E3011903811964084
:10115700118E4811AF5011CC58000011DA8574DA9E
:10116700C2DDC2DC7572007573008070800EE57198
:10117700700280560573E573700205721200268FA0
:10118700DAC2DDC2DC80558016D2DDC2DC804DC2FA
:10119700DDC2DCE5717004C2DA8041D2DA803DC27B
:1011A700DDD2DC756F048034AFDA121CF40573E509
:1011B7007370020572C2DDC2DCE5717004C2DA80A9
:1011C7001BD2DA8017AFDA121CF4C2DDD2DC756FDE
:0E11D700028009756F04C2DDC2DCD2DAC2DB11
:0B11E500D0D0D082D083D0F0D0E03218
:1019D90043910C43920CE4F5DBEF25E0F5DB301A7B
:1019E9000343DB0175DD2575DC2575D84453F8FE05
:0919F90053F7FEE4F56FD2E82279
:101BAA00E56F30E002FF22E4F570756F03EF25E080
:071BBA00F574D2DD7F022269
:101B7500E56F30E002FF22E4F5701571756F05EF32
:0B1B850025E04401F574D2DD7F022250
:061D2D0020DBFDAF6F2278
:0D0026001571AF700570747A2FF8E6FF2297
:0C1CF400747A2570F8EFF6057015712267
:0E1CB000E4F5847585FFF592F5A475A5FF2275
:0E1CBE00EE3395E0FDFC227B007A00791B22BC
:101A9900C215C217C214D2A2C2A0C2A1E4FDFF128C
:101AA9001B1DE4FD7F01121B1D7F081213FA7F0421
:031AB9000213FA1B
:101B1D00EF146011047016BD0104C2A78002D2A794
:0E1B2D00A2A7921622BD0103C2A622D2A622B2
:1013FA00EF14B40800505C90140F75F003A4C58371
:10140A0025F0C5837302142702142D021434021422
:10141A004002144202144002144C021454D21575AC
:10142A00190122C215A21692A722D217751A027D95
:10143A00017F01021B1D8005C214C28722C214D279
:10144A008722D214D28775180122C2A47F011218EA
:04145A007ED2A42278
:1017CC00301512D5190F30A707C2A775190F800550
:1017DC00D2A7751923E51AD39400400CD51A09C267
:1017EC0017E4FD7F01121B1D301411D5180E308724
:0D17FC0006C28775180522D28775181E22B7
:101ADD00C374039FFE1392A0EEA2E192A1AF80CF3B
:0F1AED005480CFED547FCF4FCF8F80C2A2D2A2B3
:011AFC0022C7
:06191C008B3B8A3C893D73
:10192200E4FCCFECCF7D20121ADD0CBC04F4E4FC05
:10193200AB3BAA3CA93D8C82758300120A47FD602D
:0B1942000ACFECCF121ADD0CBC04E54C
:01194D002277
:04127C008F828E834C
:10128000121CBEE47B0F7A27F9F8C3120BD350036C
:1012900090270FAF82AE83121CBE7B197AFC79FFB8
:1012A00078FFD3120BD3400390FC19E4F52F741B85
:1012B000252FF8E4F6052FE52FB405F2AE83AF82B3
:1012C000121CBE121CC5120E1EE51E701A752F03CD
:1012D000741A252FF8E6FF741B252FF8C6EFC6D524
:1012E0002FEE751B2080E2121CC512191C30081548
:1012F0007F811200167F181200167F02120016124C
:051300001CC5121C5089
:0113050022C5
:101B3B0046554C4C0050524F47005A4C4F47004DA6
:0D1B4B004F440076332D340054726967005A
:101A500078DCE6FE08E6FF22E6FE08E6FFE4FCFD91
:101A60002278D1120C0E78C9020C27C3E55C94B819
:051A7000E55B940B2270
:03001300021ABC12
:101ABC00C0E0C0D075D01020100CAF8DEFAD8BF501
:101ACC0058EDF559D210758D00758B00D0D0D0E043
:011ADC0032D7
:02187E008F3A9F
:10188000E4F53BF53CC3E53C953AE53B9400502339
:10189000900000AF82AE83E4FCFD7B207A4EF9F825
:1018A000D3120BD34003A380EA053CE53C70D60578
:0318B0003B80D2A8
:0118B3002212
:0E1CCC007BFF7A1B793B12191C7F0A02187EDF
:0F1C8400D20D301806121CCCC20D2212174C22A2
:05000E00C20D021844C0
:101BC10078D5120C3300000000121A6178D1120C82
:061BD100330000000022B9
:101C74008E2C8F2DEEFF120016AF2DE52D020016CF
:10003600121CB0121D0A121A997F0412187E2097FC
:10004600147BFF7A1B794012191C7D017F01121364
:1000560006D2AF80FE209612D2AF12194EC21A7F78
:10006600701219D91211F012058312194E7A1B79E2
:100076004512056E120579D2AF7BFF7A1B794A12BB
:10008600191C78B3E62430FD7F03121ADD7F0412B3
:10009600187E7A1B794E12056EC21A7F701219D914
:1000A6007F0112187E1211F0120019E4F579121868
:1000B600097F0112187EE478D9F608F612001AA212
:1000C600969209A297920AE4F52478CD120C330091
:1000D600000000E4F52578D5120C33FFFFD8F1783F
:1000E600C9120C3300000000C20B78D1120C330089
:1000F600000000C20FC213C20DC20EE4F561F56224
:10010600F526F527C208F55BF55CF558F559C210DA
:10011600F55AC211F557F556F555F554F560F55FE4
:10012600F55EF55DF52078B0E624FE600B14600CF4
:100136002402700AD2018006D2068002D20078B16B
:10014600E624FE6007047006D2028002D20778B267
:10015600E624FE600B14600C2402700AD2038006AB
:10016600D2048002D205300117C20178A8121A58AB
:100176007B64FAF9F8120AA88F578E568D558C545F
:10018600E579C3940240F9E4F579A208B392A63062
:100196000E32A209309601B3400BA20A309701B382
:1001A60040030202D530961130970EC20EE4F56177
:1001B600F5627F041213FAC20BA2969209A29792D5
:1001C6000A0202D5209605209702D21230965630A2
:1001D6009753301231C21278C9120C0EEC4D4E4FA5
:1001E60078D5700C120C3300000000121A618010D2
:1001F600120C330000000078C9120C330000000016
:10020600D20AD2098024789FE6601F0562E56270F3
:10021600020561D394B8E561940B400ED20E7F05BA
:100226001213FA8005E4F561F562A209309601B36E
:10023600502AA296920930961C201219121A6B5057
:1002460014C201300B06C20B7F068004D20B7F0757
:100256001213FA805BE4F55BF55C805420965174CA
:100266000A255CF55CE4355BF55B121A6B4041E5EB
:100276005C9410E55B94275037755B27755C1030EE
:100286000807C2081205798027D2087D01E4FF120B
:1002960013067F891200167F0112187E7F821200D4
:1002A600167F0112187E7F841200167F3112001607
:1002B600A20A309701B35017A297920A30971020DE
:1002C600120DB20D300D05121C84800312000E12A1
:1002D60007DDAF57AE56AD55AC54EC4D4E4F6026CC
:1002E60074FF2FF557EE34FFF556ED34FFF555EC58
:1002F60034FFF554AF57AE56AD55FC4D4E4F700614
:10030600200D03121C84AF60AE5FAD5EAC5DEC4D9C
:100316004E4F602374FF2FF560EE34FFF55FED342A
:10032600FFF55EEC34FFF55DAF60AE5FAD5EFC4D94
:100336004E4F700312000E2010030203E5C2AFC237
:1003460010D2AFE485592B85582AF529F528AF2B0D
:10035600AE2AAD29AC287B107A27F9F8120AA88FA5
:100366002B8E2A8D298C28E4FB7A90F9F8121641F7
:100376008F2B8E2A8D298C2878A6E66009C374B83F
:100386009FFF740B9EFEE55A14601624FE6020241F
:10039600037049C3EF94B0EE9404500E755A018071
:1003A60009D3EF9414EE94054035755A038030C393
:1003B600EF94B0EE94045027755A01300006200DD4
:1003C60003121C84300305C203121BC1300D02D276
:1003D600117BFF7A1B795312191C8003E4F55A0529
:1003E60025E525C394015003020568E4F525FB7A4B
:1003F6000079DB121A0278DCEEF608EFF678DBE617
:100406006402600302056878CD120C1AE8C0E0E9C0
:10041600C0E0EAC0E0EBC0E0121A50789EE6FD129A
:1004260015AED0E0FBD0E0FAD0E0F9D0E0F8EB2F43
:10043600FFEA3EFEE93DFDE83CFC78CD120C2705BF
:1004460024E524C39405500302056878CD120C0EEA
:10045600E47B05FAF9F812164178CD120C2778CD0F
:10046600120C0E78C9120C1AC3EF9BFFEE9AFEED22
:1004760099FDEC98FC78CD120C2778D5120C0E78E5
:10048600CD120C1AD3120BD3400A78CD120C0E786B
:10049600D5120C27300B0C78D5120C0E78DEEEF642
:1004A60008EFF678CD120C0E78DCEEF608EFF63093
:1004B6000B0308800278DCE6FE08E6FF12127C30A9
:1004C6001306121A50121C740527E527700205261A
:1004D600C3789D96E52618964038E4F526F527302C
:1004E6000F06121A50121C74300D277F031213FACE
:1004F60020181978A7E6600C3011097F007E821259
:100506001382C211121A501213828006121CCC12C8
:10051600000E78CD120C0E78D1120C2778CD120C65
:100526003300000000E4F524300405C204121BC1A8
:1005360030061678AC121A5878D1120C1AD3120B50
:10054600D34006200D03121C8430071678AE121A0B
:100556005878D1120C1AC3120BD35006300D031261
:08056600000E1217CC02018601
:10056E007BFF12191C7F0412187E2278B5E6FDE47B
:05057E00FF121306222C
:101A2A00444C0021536967005A4C4F47004D4F44BC
:101A3A0000332D34004A756E203231203230303670
:061A4A000050524F47005E
:1016C800AF34AE33AD32AC31EC4D4E4F22EF24FF88
:1016D800F534EE34FFF533ED34FFF532EC34FFF535
:1016E8003122E475342075334EF532F53122E47534
:1016F8003401F533F532F53122752E00752F00755A
:03170800309A22F2
:0F1C93007F041213FAC20BC20EE4F561F5622250
:1007DD00121CDAEF7003020A0E121B58EF120C4CAA
:1007ED0009D22409DE2A09F94809E450092A5208D8
:1007FD001B6108AC630A036808FF6C0905720902E6
:10080D0073092E7409A276099C7800000A0E121C39
:10081D00937BFF7A1A792A12191C1216EA121CDA26
:10082D00EF700A1216C860051216D580F01216C8A0
:10083D007003020A0E121B588F2D1215FAE4F534AF
:10084D001216FAE47F06FEFDFCAB34AA33A932A8DA
:10085D0031C3120BE9501F121BEC8F2D120016E540
:10086D00342401F534E43533F533E43532F532E42F
:10087D003531F53180CD121BEC8F2DE52D64806067
:10088D0016E52D64816010120016121BEC8F2D12CF
:10089D000016752C018003E4F52CE52C70D822127E
:1008AD0017011216F6F52D1216C860241216EA124B
:1008BD001CDAEF700A1216C860051216D580F012F8
:1008CD0016C86003120A0F052DE52DC3941C40D7E1
:1008DD001216C8601A789AB6AB0708B6CD0302098E
:1008ED00DB7BFF7A1A792D12191C7F0A02187E0202
:1008FD000999B20F2202145E121701E4F52DAB2EE9
:10090D000530E530AA2F7002052F14F9120A2EFFBB
:10091D00120016052DE52DC3941C40E22243A208BA
:10092D0022121C93752E00752F007530771216F656
:10093D00F52D1216C860241216EA121CDAEF700A91
:10094D001216C860051216D580F01216C860031273
:10095D000A0F052DE52DC3940240D71216C8602C41
:10096D00AE77AF78EE3395E0FDFC78D1120C1AC35B
:10097D00EF9BF538EE9AF537ED99F536EC98F535A0
:10098D00AF3878A4E537F608EFF6804202168512E7
:10099D001C930214B77A1A7932120A237A1A79370C
:1009AD00121C5078B3E62430FF120016121D1D7F65
:1009BD00761200167A1A793B120A237A1A793F12A7
:1009CD001C50021D1D121C93E478A4F608F60219A2
:1009DD00AC121C93021561121C937BFF7A1A794B92
:1009ED0012191C7D017F0112130680FE7D03E4FFA9
:1009FD00121306D2132278B5E6FDE4FF121306C2D8
:010A0D0013D5
:100A0E0022121B58AB2EAA2FA930852D827583007A
:100A1E00EF120A86227BFF121C50121D1D7BFF2235
:0A1D0A00E4F5955396BF53A27F2223
:101809005389F0438901538FFE758C70E4F58A532F
:10181900B8FD53B7FDD2A9D28C53890F4389905390
:101829008FEFF58DF58B4391105392EF53B8F75322
:0B183900B7F7D2ABD28ED28AD2AA221F
:03000B00021D14BF
:091D14000579758C70758A0032A6
:03001B00021D269D
:071D2600758D00758B003282
:101C14000D0A0030313233343536373839414243D6
:041C240044454600ED
:101C2800AF4DAB41AA42A943054D22AF40AE3FADEF
:041C38003EAC3D225F
:101306005387BF75985053877FE4F5BABF010543ED
:10131600A240800353A2BFE4F5BDED14601514602E
:101326001A14601F1460242404702575BEF075BF5E
:101336000B802375BEF075BF05801B75BEF075BFAB
:1013460002801375BE7075BF01800B75BEB0800339
:1013560075BE30E4F5BF75BD035391FE439201435C
:1013660091025392FDC21C53B8EF53B7EF43B81026
:0C137600E478C7F618F678C8F6D2AC226E
:030023000218E8D8
:1018E800C0E0C0D075D01030981E78C7E6C3940FFA
:1018F800501418E60624B6F8A69978C70618E6C361
:10190800941040027600C298309904C299C21CD043
:04191800D0D0E03219
:08000300201CFDD21C8F992284
:101AFD0078C7E6D39400401508E60624B6F8E6FF4D
:0F1B0D0078C71608E6C394104005E4F6227F005F
:011B1C0022A6
:03001600020003E2
:101B58007F207E4E78C7E67010D3EF9400EE940095
:0C1B68004007EF1F70EE1E80EB121AFD0C
:011B7400224E
:101C5000120A2EFF600C120016740129F9E43AFAF8
:031C600080EE22F1
:0E1CDA0078C7E6D3940040037F01227F0022EA
:091D1D007BFF7A1C7914021C50B2
:0E0E1E008F408E3F8D3E8C3D8B418A42894332
:100E2C00E4F54DEC4D4E4F7017E94A4B70057F3091
:100E3C00020016121C288F827583007430020F4139
:100E4C00121C35EC33502AE5434542454170077F6F
:100E5C002D120016800D121C288F82758300742DA4
:100E6C00120A86121C33120BC58F408E3F8D3E8C9E
:100E7C003D754C017547007546CA75459A75443BDE
:100E8C00E4FFFEFDFCAB47AA46A945A844D3120BD0
:100E9C00E95003020F2C121C33A844120B338F4B56
:100EAC008E4A8D498C48EC4D4E4F7004E54C7023A6
:100EBC00E54B2430FFE543454245417005120016D1
:100ECC00800EAE4D121C2A8E82758300EF120A869C
:100EDC00E4F54CAF47AE46AD45AC44AB4BAA4AA982
:100EEC0049A848120AA8CAEECAC9EDC9C8ECC8C3B9
:100EFC00E5409FF540E53F9AF53FE53E99F53EE527
:100F0C003D98F53DAF47AE46AD45AC44E47B0AFA9F
:100F1C00F9F8120B338F478E468D458C44020E8C9C
:100F2C00E542454345416010AB41AA42A943854D7A
:080F3C0082758300E4120A86AD
:010F4400228A
:100C72000134C35001DBBF68028BBB800344B798C9
:100C82000407B3B004D5AFC805A9ABE00689A7F83D
:100C92000775A410086DA02809719C400A81985814
:100CA2000B9F94700CCA90880DE98CF90E048CA0ED
:100CB2000EA88AAC0F4D88B80FF786C410A184D055
:100CC200115182DC120580E812BB7EF413747D00A0
:100CD20014307B0C14F2791815B87724168075300D
:100CE200174B733C1819714818ED6F5419C46D6095
:100CF2001AA16B6C1B7E69781C6167841D4A659022
:100D02001E37639C1F2561A8201A5FB421125DC0A3
:100D1200220D5BCC230E59D8241557E4251F55F01C
:100D2200262F53FC27425208285B501429764E2066
:100D32002A9B4C2C2BC04A382CEE48442E1E46507F
:100D42002F55445C308F426831D1407433173E8056
:100D520034633C8C35B13A98370938A4386636B0DA
:100D620039C734BC3B2D32C83C9D30D43E0F2EE0F7
:100D72003F882CEC41062AF8428D2904441827109A
:100D820045AB251C4741232848E121344A861F40B0
:100D92004C311D4C4DE21B584F9C1964515D17702C
:100DA2005323157C54EF138856C4119458A20FA0F4
:100DB2005A830DAC5C6D0BB85E6009C4605807D0F5
:100DC200625A05DC646203E8667301F4688A000013
:100DD2006AA1FE0C6CB8FC186ECFFA2470E6F830EB
:100DE2000000000000000000000000000000000001
:100DF20000000000000000000000000000000000F1
:100E020000000000000000000000000000000000E0
:0C0E1200000000000000000000000000D4
:10178D0075F004E533A42472F582E5F0340CF5838D
:10179D00E49322FE740193FF75F004E533A422F562
:1017AD0083C37401939FFFE4939EFEE4228F348ED6
:0F17BD00338D328C31228F308E2F8D2E8C2D223A
:101C3C00C3EF9DEE9C400AD3EF9BEE9A50037F01BD
:041C4C00227F0022D1
:040F45008E318F3228
:100F4900E4F53312178DFC740193FD1217A524766D
:100F5900F582E5F0340CF583E493FA740193FBAF61
:100F690032AE31121C3CEF700302103512178D128C
:100F790017A02476F582E5F0340C1217AC8F378E62
:100F890036F535F5341217A52478F582E5F0340CD9
:100F9900F583E4931217A02474F582E5F0340C125A
:100FA90017AC8F3B8E3AF539F538AD39AC38120BA1
:100FB900C58F3B8E3A8D398C38AE31AF32E4FCFDAA
:100FC900EEC0E0EFC0E012178DFE740193FBCAEE8C
:100FD900CAD0E0FFD0E0FEC3EF9BFFEE9AFEED948E
:100FE90000FDEC9400FCAB3BAA3AA939A838120AD7
:100FF900A8AB37AA36A935A834121641C8ECC8C916
:10100900EDC9CAEECACBEFCB1217A52474F582E558
:10101900F0340CF583E493FE740193FFE4FCFDEBDB
:101029002FFFEA3EFEED39FDEC38FC220533E533AE
:0D103900C3946A5003020F4CE4FFFEFDFC5F
:011046002287
:01001A0022C3
:10150F001217BAAB34AA33A932A831E8C0E078A2D7
:10151F00E6FE08E6FFE4FCFDD0E0F8120AA8121779
:10152F00BA780E120BFA1217BA78A4E6FE08E6FF85
:10153F00EE3395E0FDFCE5342FF534E5333EF5331E
:10154F00E5323DF532E5313CF531AF34AE33AD32F6
:02155F00FC226C
:0215AE008D2C82
:1015B000120F451217C312150F1217C3E52C146032
:1015C0001C14702DE47FE87E03FDFCAB30AA2FA92C
:1015D0002EA82D120AA8E47BE87A0B800CAF30AE5F
:1015E0002FAD2EAC2DE47B03FAF9F8121641121739
:0915F000C3AF30AE2FAD2EAC2DBF
:0115F90022CF
:100A2E00BB010689828A83E0225002E722BBFE02C6
:090A3E00E32289828A83E49322F9
:100A4700BB010CE58229F582E5833AF583E0225064
:100A570006E92582F8E622BBFE06E92582F8E222AE
:0D0A6700E58229F582E5833AF583E49322C8
:100A7400BB010689828A83F0225002F722BBFE0161
:020A8400F3225B
:100A8600F8BB010DE58229F582E5833AF583E8F0A6
:100A9600225006E92582C8F622BBFE05E92582C852
:020AA600F2223A
:100AA800E88FF0A4CC8BF0A42CFCE98EF0A42CFCED
:100AB8008AF0EDA42CFCEA8EF0A4CDA8F08BF0A46B
:100AC8002DCC3825F0FDE98FF0A42CCD35F0FCEBCA
:100AD8008EF0A4FEA9F0EB8FF0A4CFC5F02ECD398F
:0F0AE800FEE43CFCEAA42DCE35F0FDE43CFC22FC
:100AF70075F008758200EF2FFFEE33FECD33CDCCB6
:100B070033CCC58233C5829BED9AEC99E582984038
:100B17000CF582EE9BFEED9AFDEC99FC0FD5F0D615
:100B2700E4CEFBE4CDFAE4CCF9A88222B800C1B93F
:100B37000059BA002DEC8BF084CFCECDFCE5F0CB7D
:100B4700F97818EF2FFFEE33FEED33FDEC33FCEBB6
:100B570033FB10D703994004EB99FB0FD8E5E4F971
:100B6700FA227818EF2FFFEE33FEED33FDEC33FC5E
:100B7700C933C910D7059BE99A4007EC9BFCE99A52
:100B8700F90FD8E0E4C9FAE4CCFB2275F010EF2F97
:100B9700FFEE33FEED33FDCC33CCC833C810D70797
:100BA7009BEC9AE899400AED9BFDEC9AFCE899F8D2
:0E0BB7000FD5F0DAE4CDFBE4CCFAE4C8F92265
:10164100C2D5E830E70FB2D5E4C39BFBE49AFAE4D4
:1016510099F9E498F8EC30E717B2D5121677120B26
:1016610033E4C39BFBE49AFAE499F9E498F8800324
:10167100120B3330D50DE4C39FFFE49EFEE49DFDC4
:04168100E49CFC22C7
:0E0BC500C3E49FFFE49EFEE49DFDE49CFC2241
:100BD300EB9FF5F0EA9E42F0E99D42F0EC6480C899
:060BE30064809845F02239
:100BE900EB9FF5F0EA9E42F0E99D42F0E89C45F062
:010BF90022D9
:100BFA00E86010ECA2E713FCED13FDEE13FEEF1311
:040C0A00FFD8F022FD
:0C0C0E00E6FC08E6FD08E6FE08E6FF2212
:0D0C1A00E6FB08E6F908E6FA08E6CBF8224A
:0C0C2700ECF608EDF608EEF608EFF622F9
:100C3300D083D082E493F608740193F60874029388
:090C4300F608740393F6740473BF
:100C4C00D083D082F8E4937012740193700DA3A337
:100C5C0093F8740193F5828883E47374029368604B
:060C6C00EFA3A3A380DF4B
:00000001FF
